:020000040000FA
:10000000052800000000000000008501860183161D
:100010009B010F178F1607309C0085018601831204
:10002000FF308500860018208501860118201028E1
:100030000330A2008930A100A00B1C28A10B1C28B2
:10004000A20B1C280800FF3FFF3FFF3FFF3FFF3F81
:10005000FF3FFF3FFF3FFF3FFF3FFF3FFF3FFF3FB0
:10006000FF3FFF3FFF3FFF3FFF3FFF3FFF3FFF3FA0
:10007000FF3FFF3FFF3FFF3FFF3FFF3FFF3FFF3F90
:10008000FF3FFF3FFF3FFF3FFF3FFF3FFF3FFF3F80
:04400E00303FFF3F01
:08400000FF3FFF3FFF3FFF3FC0
:00000001FF
